:101A240033302E322020200008000803080608095D
:101A3400080C080F081208150819081C081F0822AA
:101A440008250828082B082F083208350838083BD1
:101A5400083E084108450848084B084E08510854F8
:101A64000857085B085E086108640867086A086D1F
:101A7400087108740877087A087D08800883088646
:101A8400088A088D0890089308960899089C08A06D
:101A940008A308A608A908AC08AF08B208B508B995
:101AA40008BC08BF08C208C508C808CB08CE08D2BD
:101AB40008D508D808DB08DE08E108E408E708EBE5
:101AC40008EE08F108F408F708FA08FD090009040B
:101AD4000907090A090D0910091309160919091C2E
:101AE4000920092309260929092C092F0932093556
:101AF4000938093C093F094209450948094B094E7F
:101B0400095109540957095B095E096109640967A8
:101B1400096A096D0970097309760979097D0980D3
:101B2400098309860989098C098F099209950998FD
:101B3400099B099E09A209A509A809AB09AE09B127
:101B440009B409B709BA09BD09C009C309C609C955
:101B540009CC09D009D309D609D909DC09DF09E27E
:101B640009E509E809EB09EE09F109F409F709FAAD
:101B740009FD0A000A030A060A090A0D0A100A13D3
:101B84000A160A190A1C0A1F0A220A250A280A2BFD
:101B94000A2E0A310A340A370A3A0A3D0A400A432D
:101BA4000A460A490A4C0A4F0A520A550A580A5B5D
:101BB4000A5E0A610A640A670A6A0A6D0A700A738D
:101BC4000A760A790A7C0A7F0A820A850A880A8BBD
:101BD4000A8E0A910A940A970A9A0A9D0AA00AA3ED
:101BE4000AA60AA90AAC0AAE0AB10AB40AB70ABA22
:101BF4000ABD0AC00AC30AC60AC90ACC0ACF0AD255
:101C04000AD50AD80ADB0ADE0AE10AE30AE60AE987
:101C14000AEC0AEF0AF20AF50AF80AFB0AFE0B01BB
:101C24000B040B070B090B0C0B0F0B120B150B18EA
:101C34000B1B0B1E0B210B240B260B290B2C0B2F20
:101C44000B320B350B380B3B0B3D0B400B430B4658
:101C54000B490B4C0B4F0B510B540B570B5A0B5D91
:101C64000B600B630B650B680B6B0B6E0B710B74CA
:101C74000B760B790B7C0B7F0B820B850B870B8A06
:101C84000B8D0B900B930B950B980B9B0B9E0BA141
:101C94000BA40BA60BA90BAC0BAF0BB10BB40BB77E
:101CA4000BBA0BBD0BBF0BC20BC50BC80BCA0BCDBC
:101CB4000BD00BD30BD60BD80BDB0BDE0BE10BE3FA
:101CC4000BE60BE90BEB0BEE0BF10BF40BF60BF93C
:101CD4000BFC0BFF0C010C040C070C090C0C0C0F77
:101CE4000C120C140C170C1A0C1C0C1F0C220C24B8
:101CF4000C270C2A0C2D0C2F0C320C350C370C3AFB
:101D04000C3D0C3F0C420C450C470C4A0C4C0C4F40
:101D14000C520C540C570C5A0C5C0C5F0C620C6487
:101D24000C670C690C6C0C6F0C710C740C770C79CF
:101D34000C7C0C7E0C810C840C860C890C8B0C8E18
:101D44000C900C930C960C980C9B0C9D0CA00CA264
:101D54000CA50CA80CAA0CAD0CAF0CB20CB40CB7AF
:101D64000CB90CBC0CBE0CC10CC30CC60CC90CCBFE
:101D74000CCE0CD00CD30CD50CD80CDA0CDD0CDF4B
:101D84000CE20CE40CE70CE90CEB0CEE0CF00CF39D
:101D94000CF50CF80CFA0CFD0CFF0D020D040D07EC
:101DA4000D090D0B0D0E0D100D130D150D180D1A3B
:101DB4000D1C0D1F0D210D240D260D280D2B0D2D91
:101DC4000D300D320D340D370D390D3C0D3E0D40E7
:101DD4000D430D450D470D4A0D4C0D4E0D510D5340
:101DE4000D560D580D5A0D5D0D5F0D610D640D6698
:101DF4000D680D6A0D6D0D6F0D710D740D760D78F6
:101E04000D7B0D7D0D7F0D810D840D860D880D8A52
:101E14000D8D0D8F0D910D940D960D980D9A0D9DB0
:101E24000D9F0DA10DA30DA50DA80DAA0DAC0DAE12
:101E34000DB10DB30DB50DB70DB90DBC0DBE0DC073
:101E44000DC20DC40DC60DC90DCB0DCD0DCF0DD1D9
:101E54000DD30DD60DD80DDA0DDC0DDE0DE00DE23F
:101E64000DE50DE70DE90DEB0DED0DEF0DF10DF3A6
:101E74000DF50DF70DFA0DFC0DFE0E000E020E040D
:101E84000E060E080E0A0E0C0E0E0E100E120E1476
:101E94000E160E180E1B0E1D0E1F0E210E230E25E0
:101EA4000E270E290E2B0E2D0E2F0E310E330E354E
:101EB4000E370E390E3B0E3C0E3E0E400E420E44C3
:101EC4000E460E480E4A0E4C0E4E0E500E520E5436
:101ED4000E560E580E5A0E5B0E5D0E5F0E610E63AB
:101EE4000E650E670E690E6B0E6C0E6E0E700E7222
:101EF4000E740E760E780E790E7B0E7D0E7F0E819B
:101F04000E830E840E860E880E8A0E8C0E8E0E8F15
:101F14000E910E930E950E960E980E9A0E9C0E9E92
:101F24000E9F0EA10EA30EA50EA60EA80EAA0EAC11
:101F34000EAD0EAF0EB10EB20EB40EB60EB80EB993
:101F44000EBB0EBD0EBE0EC00EC20EC30EC50EC716
:101F54000EC80ECA0ECC0ECD0ECF0ED10ED20ED49C
:101F64000ED60ED70ED90EDB0EDC0EDE0EDF0EE122
:101F74000EE30EE40EE60EE70EE90EEA0EEC0EEEAC
:101F84000EEF0EF10EF20EF40EF50EF70EF90EFA38
:101F94000EFC0EFD0EFF0F000F020F030F050F06C0
:101FA4000F080F090F0B0F0C0F0E0F0F0F110F124D
:101FB4000F140F150F160F180F190F1B0F1C0F1EE0
:101FC4000F1F0F210F220F230F250F260F280F2974
:101FD4000F2A0F2C0F2D0F2F0F300F310F330F340B
:101FE4000F350F370F380F3A0F3B0F3C0F3E0F3FA3
:101FF4000F400F420F430F440F450F470F480F493F
:102004000F4B0F4C0F4D0F4F0F500F510F520F54DA
:102014000F550F560F570F590F5A0F5B0F5C0F5E7A
:102024000F5F0F600F610F620F640F650F660F671C
:102034000F680F6A0F6B0F6C0F6D0F6E0F6F0F71C0
:102044000F720F730F740F750F760F770F790F7A66
:102054000F7B0F7C0F7D0F7E0F7F0F800F810F8210
:102064000F840F850F860F870F880F890F8A0F8BB8
:102074000F8C0F8D0F8E0F8F0F900F910F920F9368
:102084000F940F950F960F970F980F990F9A0F9B18
:102094000F9C0F9D0F9E0F9F0FA00FA10FA20FA3C8
:1020A4000FA40FA50FA50FA60FA70FA80FA90FAA7E
:1020B4000FAB0FAC0FAD0FAE0FAE0FAF0FB00FB134
:1020C4000FB20FB30FB40FB40FB50FB60FB70FB8ED
:1020D4000FB90FB90FBA0FBB0FBC0FBD0FBD0FBEA9
:1020E4000FBF0FC00FC10FC10FC20FC30FC40FC466
:1020F4000FC50FC60FC70FC70FC80FC90FCA0FCA26
:102104000FCB0FCC0FCC0FCD0FCE0FCE0FCF0FD0E8
:102114000FD00FD10FD20FD20FD30FD40FD40FD5AE
:102124000FD60FD60FD70FD80FD80FD90FD90FDA74
:102134000FDB0FDB0FDC0FDC0FDD0FDD0FDE0FDF3E
:102144000FDF0FE00FE00FE10FE10FE20FE20FE30B
:102154000FE30FE40FE40FE50FE50FE60FE60FE7DB
:102164000FE70FE80FE80FE90FE90FEA0FEA0FEBAB
:102174000FEB0FEC0FEC0FEC0FED0FED0FEE0FEE7E
:102184000FEF0FEF0FEF0FF00FF00FF00FF10FF154
:102194000FF20FF20FF20FF30FF30FF30FF40FF42C
:1021A4000FF40FF50FF50FF50FF60FF60FF60FF707
:1021B4000FF70FF70FF70FF80FF80FF80FF80FF9E5
:1021C4000FF90FF90FF90FFA0FFA0FFA0FFA0FFBC5
:1021D4000FFB0FFB0FFB0FFB0FFC0FFC0FFC0FFCA7
:1021E4000FFC0FFD0FFD0FFD0FFD0FFD0FFD0FFD8C
:1021F4000FFE0FFE0FFE0FFE0FFE0FFE0FFE0FFE73
:102204000FFF0FFF0FFF0FFF0FFF0FFF0FFF0FFF5A
:102214000FFF0FFF0FFF0FFF0FFF0FFF0FFF0FFF4A
:102224000FFF0FFF0FFF0FFF0FFF0FFF0FFF0FFF3A
:102234000FFF0FFF0FFF0FFF0FFF0FFF0FFF0FFF2A
:102244000FFF0FFF0FFF0FFF0FFF0FFF0FFF0FFF1A
:102254000FFF0FFE0FFE0FFE0FFE0FFE0FFE0FFE11
:102264000FFE0FFD0FFD0FFD0FFD0FFD0FFD0FFD09
:102274000FFC0FFC0FFC0FFC0FFC0FFB0FFB0FFB05
:102284000FFB0FFB0FFA0FFA0FFA0FFA0FF90FF902
:102294000FF90FF90FF80FF80FF80FF80FF70FF702
:1022A4000FF70FF70FF60FF60FF60FF50FF50FF503
:1022B4000FF40FF40FF40FF30FF30FF30FF20FF209
:1022C4000FF20FF10FF10FF00FF00FF00FEF0FEF10
:1022D4000FEF0FEE0FEE0FED0FED0FEC0FEC0FEC19
:1022E4000FEB0FEB0FEA0FEA0FE90FE90FE80FE826
:1022F4000FE70FE70FE60FE60FE50FE50FE40FE436
:102304000FE30FE30FE20FE20FE10FE10FE00FE045
:102314000FDF0FDF0FDE0FDD0FDD0FDC0FDC0FDB58
:102324000FDB0FDA0FD90FD90FD80FD80FD70FD66D
:102334000FD60FD50FD40FD40FD30FD20FD20FD186
:102344000FD00FD00FCF0FCE0FCE0FCD0FCC0FCCA1
:102354000FCB0FCA0FCA0FC90FC80FC70FC70FC6BD
:102364000FC50FC40FC40FC30FC20FC10FC10FC0DD
:102374000FBF0FBE0FBD0FBD0FBC0FBB0FBA0FB900
:102384000FB90FB80FB70FB60FB50FB40FB40FB323
:102394000FB20FB10FB00FAF0FAE0FAE0FAD0FAC4A
:1023A4000FAB0FAA0FA90FA80FA70FA60FA50FA574
:1023B4000FA40FA30FA20FA10FA00F9F0F9E0F9D9D
:1023C4000F9C0F9B0F9A0F990F980F970F960F95CD
:1023D4000F940F930F920F910F900F8F0F8E0F8DFD
:1023E4000F8C0F8B0F8A0F890F880F870F860F852D
:1023F4000F840F820F810F800F7F0F7E0F7D0F7C64
:102404000F7B0F7A0F790F770F760F750F740F7399
:102414000F720F710F6F0F6E0F6D0F6C0F6B0F6AD2
:102424000F680F670F660F650F640F620F610F600F
:102434000F5F0F5E0F5C0F5B0F5A0F590F570F564C
:102444000F550F540F520F510F500F4F0F4D0F4C8C
:102454000F4B0F490F480F470F450F440F430F42CF
:102464000F400F3F0F3E0F3C0F3B0F3A0F380F3713
:102474000F350F340F330F310F300F2F0F2D0F2C5B
:102484000F2A0F290F280F260F250F230F220F21A4
:102494000F1F0F1E0F1C0F1B0F190F180F160F15F0
:1024A4000F140F120F110F0F0F0E0F0C0F0B0F093C
:1024B4000F080F060F050F030F020F000EFF0EFD8E
:1024C4000EFC0EFA0EF90EF70EF50EF40EF20EF1E6
:1024D4000EEF0EEE0EEC0EEA0EE90EE70EE60EE43B
:1024E4000EE30EE10EDF0EDE0EDC0EDB0ED90ED790
:1024F4000ED60ED40ED20ED10ECF0ECD0ECC0ECAE9
:102504000EC80EC70EC50EC30EC20EC00EBE0EBD43
:102514000EBB0EB90EB80EB60EB40EB20EB10EAF9F
:102524000EAD0EAC0EAA0EA80EA60EA50EA30EA1FD
:102534000E9F0E9E0E9C0E9A0E980E960E950E935E
:102544000E910E8F0E8E0E8C0E8A0E880E860E84C1
:102554000E830E810E7F0E7D0E7B0E790E780E7625
:102564000E740E720E700E6E0E6C0E6B0E690E678C
:102574000E650E630E610E5F0E5D0E5B0E5A0E58F5
:102584000E560E540E520E500E4E0E4C0E4A0E485F
:102594000E460E440E420E400E3E0E3C0E3B0E39CD
:1025A4000E370E350E330E310E2F0E2D0E2B0E2937
:1025B4000E270E250E230E210E1F0E1D0E1B0E18A8
:1025C4000E160E140E120E100E0E0E0C0E0A0E081F
:1025D4000E060E040E020E000DFE0DFC0DFA0DF794
:1025E4000DF50DF30DF10DEF0DED0DEB0DE90DE70F
:1025F4000DE50DE20DE00DDE0DDC0DDA0DD80DD686
:102604000DD30DD10DCF0DCD0DCB0DC90DC60DC400
:102614000DC20DC00DBE0DBC0DB90DB70DB50DB37A
:102624000DB10DAE0DAC0DAA0DA80DA50DA30DA1F8
:102634000D9F0D9D0D9A0D980D960D940D910D8F76
:102644000D8D0D8A0D880D860D840D810D7F0D7DF8
:102654000D7B0D780D760D740D710D6F0D6D0D6A7A
:102664000D680D660D640D610D5F0D5D0D5A0D58FD
:102674000D560D530D510D4E0D4C0D4A0D470D4584
:102684000D430D400D3E0D3C0D390D370D340D320B
:102694000D300D2D0D2B0D280D260D240D210D1F94
:1026A4000D1C0D1A0D180D150D130D100D0E0D0B1F
:1026B4000D090D070D040D020CFF0CFD0CFA0CF8AE
:1026C4000CF50CF30CF00CEE0CEB0CE90CE70CE441
:1026D4000CE20CDF0CDD0CDA0CD80CD50CD30CD0CE
:1026E4000CCE0CCB0CC90CC60CC30CC10CBE0CBC60
:1026F4000CB90CB70CB40CB20CAF0CAD0CAA0CA8F2
:102704000CA50CA20CA00C9D0C9B0C980C960C9385
:102714000C900C8E0C8B0C890C860C840C810C7E1A
:102724000C7C0C790C770C740C710C6F0C6C0C69B0
:102734000C670C640C620C5F0C5C0C5A0C570C5448
:102744000C520C4F0C4C0C4A0C470C450C420C3FE1
:102754000C3D0C3A0C370C350C320C2F0C2D0C2A7A
:102764000C270C240C220C1F0C1C0C1A0C170C1418
:102774000C120C0F0C0C0C090C070C040C010BFFB5
:102784000BFC0BF90BF60BF40BF10BEE0BEB0BE95B
:102794000BE60BE30BE10BDE0BDB0BD80BD60BD3F9
:1027A4000BD00BCD0BCA0BC80BC50BC20BBF0BBD9B
:1027B4000BBA0BB70BB40BB10BAF0BAC0BA90BA63D
:1027C4000BA40BA10B9E0B9B0B980B950B930B90DF
:1027D4000B8D0B8A0B870B850B820B7F0B7C0B7984
:1027E4000B760B740B710B6E0B6B0B680B650B6329
:1027F4000B600B5D0B5A0B570B540B510B4F0B4CCF
:102804000B490B460B430B400B3D0B3B0B380B3575
:102814000B320B2F0B2C0B290B260B240B210B1E1D
:102824000B1B0B180B150B120B0F0B0C0B090B07C7
:102834000B040B010AFE0AFB0AF80AF50AF20AEF76
:102844000AEC0AE90AE60AE30AE10ADE0ADB0AD824
:102854000AD50AD20ACF0ACC0AC90AC60AC30AC0D0
:102864000ABD0ABA0AB70AB40AB10AAE0AAC0AA97E
:102874000AA60AA30AA00A9D0A9A0A970A940A9128
:102884000A8E0A8B0A880A850A820A7F0A7C0A79D8
:102894000A760A730A700A6D0A6A0A670A640A6188
:1028A4000A5E0A5B0A580A550A520A4F0A4C0A4938
:1028B4000A460A430A400A3D0A3A0A370A340A31E8
:1028C4000A2E0A2B0A280A250A220A1F0A1C0A1998
:1028D4000A160A130A100A0D0A090A060A030A004C
:1028E40009FD09FA09F709F409F109EE09EB09E808
:1028F40009E509E209DF09DC09D909D609D309D0B8
:1029040009CC09C909C609C309C009BD09BA09B76F
:1029140009B409B109AE09AB09A809A509A2099E20
:10292400099B099809950992098F098C09890986D7
:1029340009830980097D0979097609730970096D8C
:10294400096A096709640961095E095B0957095441
:102954000951094E094B094809450942093F093CF7
:10296400093809350932092F092C092909260923AF
:102974000920091C0919091609130910090D090A66
:1029840009070904090008FD08FA08F708F408F122
:1029940008EE08EB08E708E408E108DE08DB08D8DD
:1029A40008D508D208CE08CB08C808C508C208BF95
:1029B40008BC08B908B508B208AF08AC08A908A64D
:1029C40008A308A0089C0899089608930890088D05
:1029D400088A088608830880087D087A08770874BE
:1029E4000871086D086A086708640861085E085B76
:1029F400085708540851084E084B08480845084130
:102A0400083E083B083808350832082F082B0828E8
:102A140008250822081F081C081908150812080FA1
:102A2400080C0809080608031000100B10161021E2
:102A3400102C10371043104E105910651070107B75
:102A440010871092109E10A910B510C010CC10D889
:102A540010E310EF10FB11071113111E112A113688
:102A64001142114E115A11661172117E118A119779
:102A740011A311AF11BB11C811D411E011ED11F95B
:102A840012061212121F122B123812451251125E24
:102A9400126B127812841291129E12AB12B812C5E4
:102AA40012D212DF12EC12F9130613141321132E8F
:102AB400133C1349135613641371137F138C139A25
:102AC40013A713B513C313D013DE13EC13FA1408AE
:102AD400141614231431143F144E145C146A14781D
:102AE4001486149414A314B114BF14CE14DC14EB80
:102AF40014F91508151615251534154215511560C8
:102B0400156F157E158D159C15AB15BA15C915D8FD
:102B140015E715F616051615162416331643165220
:102B2400166216711681169016A016B016C016CF2E
:102B340016DF16EF16FF170F171F172F173F174F24
:102B4400175F17701780179017A117B117C117D205
:102B540017E217F3180418141825183618471857CD
:102B640018681879188A189B18AC18BE18CF18E082
:102B740018F119021914192519371948195A196B1A
:102B8400197D198F19A019B219C419D619E819FA9F
:102B94001A0C1A1E1A301A421A551A671A791A8B05
:102BA4001A9E1AB01AC31AD51AE81AFB1B0E1B2058
:102BB4001B331B461B591B6C1B7F1B921BA51BB88D
:102BC4001BCC1BDF1BF21C061C191C2D1C401C54A7
:102BD4001C671C7B1C8F1CA31CB71CCB1CDF1CF3A9
:102BE4001D071D1B1D2F1D431D581D6C1D801D958C
:102BF4001DA91DBE1DD31DE71DFC1E111E261E3B57
:102C04001E501E651E7A1E8F1EA41EB91ECF1EE402
:102C14001EFA1F0F1F251F3A1F501F661F7B1F918F
:102C24001FA71FBD1FD31FE90A00090008000700E2
:0E2C340006000500040003000200010000007D
:1034AD004102A44EC1004102A3004102A00041020D
:1034BD00A5004102B5004102980142029D00014163
:1034CD0002B001C101C10241029F06420264000027
:1034DD00410266004202B100004202B30000420206
:0C34ED009900144202B6000041029C014C
:10385E0053E3DF75B61043E32075AB80E4FF0FEF43
:10386E00B414FB43ABC0E5AB30E5FB75A90275B2F2
:01387E0087C2
:01387F002226
:10394400758850758922758E04758C5C758D5675D5
:0E395400C804E4F5CA75CBFEF5CC75CDFE2295
:1019FC0075BC9090029FE0F5BB75E88075BAF72234
:073AC60075B9F675B5F42295
:043AEE00E4F5D12208
:10399D0075E10575E2C075A48075F2C075F3FFE49D
:0C39AD00F5D675A63875D40375D5FF2239
:083AAE0043E608D2ADD2AB22C1
:1039ED00E4F58812385E12399D1239441219FC1211
:0839FD003AC6123AEE023AAE9E
:10134D00C20853D9BF1239EDA2A292089002A4305F
:10135D000805744EF08003744FF09002A4E0FF1264
:10136D003A7843F601123A1D1237C5E58054409084
:10137D0002B5F0D2AF3001081231D2C2011239805C
:10138D003002051208A7C2027B017A0279B8123722
:10139D0099EF60E19002BAE0120EDA1416041463AC
:1013AD000513D81413C71613D01713DD1A13FF1B0B
:1013BD00140A1D14101E000014B69002A37401F03F
:1013CD000214B6E49002A3F00214B6D2000214B6D1
:1013DD007B017A0279B89002C8EBF0A3EAF0A3E999
:1013ED00F0120D74FE9002A4E0FF6E60030214B6BD
:1013FD0080059002A4E0FF1238E40214B6123ADB25
:10140D000214B6123AE80214B67B017A0279B8904A
:10141D0002CBEBF0A3EAF0A3E9F0900003120D8DDF
:10142D00FF9002A4E06F60030214B69002A3E06087
:10143D00709002CBEBF0A3EAF0A3E9F09000051257
:10144D000D8DFF900006120D8DFD900004120D8D77
:10145D00FB123282804B7B017A0279B89002CBEB82
:10146D00F0A3EAF0A3E9F0900003120D8DFF9002B6
:10147D00A4E06F70349002A3E060269002CBEBF0F5
:10148D00A3EAF0A3E9F0900005120D8DFF90000680
:10149D00120D8DFD900004120D8DFB123068123768
:1014AD00C59002A4E0FF1239259002A3E07003025B
:1014BD0013959002BAE014603424FA60531470034B
:1014CD0002156B24066003021395123A4C7B017AC8
:1014DD000279B89002C8EBF0A3EAF0A3E9F090000E
:1014ED0003120D8D9002E5F0123ABE806B123A4C4C
:1014FD007B017A0279B89002C8EBF0A3EAF0A3E978
:10150D00F0900003120D8D9002E5F01237C5804862
:10151D00123A4C7B017A0279B89002CEEBF0A3EA35
:10152D00F0A3E9F0900003120D8DFF900004120D51
:10153D008DFD900005120D8DFBC0039002CEE0FBDA
:10154D00A3E0FAA3E0F9900006120D8D9002F5F0DC
:10155D00D00312311E1237C5123A9A021395123A60
:10156D004C7B017A0279B89002CEEBF0A3EAF0A39E
:10157D00E9F0900003120D8DFF900004120D8DFD0A
:10158D00900005120D8DFB12173B1237C5123A9ABA
:03159D00021395A1
:0E3A5D00E50824FFB392A4E50824FF92A322FB
:1031D2009002B5E0900298F0E58054409002B5F07C
:1031E200E07042C3900264E09408500EA3E004F041
:1031F2007059900264E004F08051A200E433FF9021
:103202000266E070047E0180027E00EE5F600E9036
:1032120002A4E0FF7BFF7A1A792412352490026619
:103222007401F08026E4900264F0A3F0900298E02A
:103232007014900266E0700EE50870047F0180024F
:103242007F008F08D207E4900266F09002A0E0901F
:1032520002A5F0E5A054409002A0F09002A5E06023
:103262001E9002A0E070189002A5F020000A9002C1
:0F327200E5F0123ABEC207229002A3E06401F019
:01328100222A
:031A0C00022F9F07
:102F9F00C0E0C083C082C0D075D000C000C006C0E2
:012FAF00071A
:102FB0009002B1E0FEA3E0F596EEF5979002A1E055
:102FC000FEA3E0FFC374FF9F9002B4F0740F9E90C5
:102FD00002B3F0E0FEA3E0F5F4EEF5F59002B6E002
:102FE000C4F854F0C868FEA3E0C4540F48FFEE5480
:102FF0000FFEC3648094885021EF25E0FFEE33FE7E
:10300000742C2FF582741A3EF583E493FF740193B8
:103010009002B1CFF0A3EFF0802BEE5407FEEF2526
:10302000E0FFEE33FE742C2FF582741A3EF583E434
:1030300093FE740193FFC374FF9F9002B2F0740F6C
:103040009E9002B1F0900299E0FEA3E0FF9002B7DB
:09305000E02FF09002B6E03EF022
:0F305900D007D006D000D0D0D082D083D0E032C4
:031A12000236F2A7
:1036F200C0E0C0F0C083C082C0D075D000C000C09E
:1037020001C002C003C004C005C006C00753C87F81
:10371200123962D007D006D005D004D003D002D02F
:0E37220001D000D0D0D082D083D0F0D0E032E1
:1039620090029FE0F5BBE004F0E0D36480949040C5
:0E397200097406F0123A5D123ACD43E81022B5
:073ACD00E50824FF928722A7
:031A210002358407
:10358400C0E0C083C082C0D075D000C004C005C0F4
:0335940006C00767
:1035970053E8DFADBDAFBEEFFE7C00E42DFFEC3E90
:1035A700FEADBBED25E02468F582E43402F583EE39
:0F35B700F0A3EFF090029FE0B41002D202D20115
:1035C600D007D006D005D004D0D0D082D083D0E0AA
:0135D60032C2
:1008A70090027EE0FFA3E09002A6CFF0A3EFF090C6
:1008B7000280E0FFA3E09002A8CFF0A3EFF0900240
:1008C70082E0FFA3E09002AACFF0A3EFF0900284AA
:1008D700E0FFA3E09002ACCFF0A3EFF0900286E038
:1008E700FFA3E09002AECFF0A3EFF090029CE06090
:1008F700509002A6E0FFA3E090031DCFF0A3EFF016
:100907009002A8E0FFA3E090031FCFF0A3EFF090C1
:1009170002AAE0FFA3E0900321CFF0A3EFF090023B
:10092700ACE0FFA3E0900323CFF0A3EFF09002AE7B
:10093700E0FFA3E0900325CFF0A3EFF0E490029C43
:10094700F07F0012102B7F0112102B7F0212102B49
:100957007F0312102B7F0412102BAF0CAE0BD37436
:10096700649F74089E5009EF249CFFEE34F78022A1
:10097700C3749C9F74079E5012C3EF9464EE94084F
:100987005009E49002D9F0A3F0800EEF2464FFEE43
:1009970034F89002D9F0A3EFF090027AE0FFA3E0D9
:1009A7009002DDCFF0A3EFF0900278E0FEA3E0FF26
:1009B700EE3395E0FDFCE42FFFEE34F8FEED34FF57
:1009C700FDEC34FFFC9002DF120E919002D9E0FE9D
:1009D700A3E0FBAA06EA3395E0F9F89002DDE0FE12
:1009E700A3E0FFEE3395E0FDFC120E2C9002D1122E
:1009F7000E91E4FB7A08F9F89002D1E0FCA3E0FD40
:100A0700A3E0FEA3E0FF1236AE9002D5120E91AE20
:100A170009AF0AE4FCFD9002DFE0F8A3E0F9A3E0E8
:100A2700FAA3E0FB120E2C9002D1120E91E4FB7A8E
:100A370020F9F89002D1E0FCA3E0FDA3E0FEA3E0DB
:100A4700FF1236AE9002DBEEF0A3EFF0AE0DAF0E65
:100A57007C007D0A120DEEE4FD9002D1120E91E4A6
:100A67007B0BFAF9F89002D1E0FCA3E0FDA3E0FECE
:100A7700A3E0FF1236AEAB07AA069002D5A3A3E008
:100A8700FEA3E02BFFEE3AFE90029DF0A3EFF0D31A
:100A970094FFEE6480948F400A90029D740FF0A338
:100AA70074FFF0C390029EE0940190029DE0648081
:100AB70094805005E4F0A304F090029DE0FEA3E0CB
:100AC700FFEE3395E0FDFCE4FB7A0BF9F8120E2CF0
:100AD7009002D1120E919002D1E0FCA3E0FDA3E0B9
:100AE700FEA3E0FFE4FB7A10F9F81236AE9002D1CC
:100AF700120E919002D5120E9D00000000E47F0BAC
:100B0700FEFDFC9002D5E0F8A3E0F9A3E0FAA3E02C
:100B1700FBC3120E7B4003020BB79002D5A3A3E0E1
:100B2700FEA3E0902C2C75F002120ECEEE25E025E8
:100B370083F583E493FE740193FF9002D9EEF0A34B
:100B4700EFF0EE3395E0FDFC9002D1E0F8A3E0F979
:100B5700A3E0FAA3E0FBC3120E7B402C9002D1A3C3
:100B6700A3E0FEA3E0FF9002D9E0FCA3E0FDEF9D28
:100B7700FFEE9C9002E3F0A3EFF09002D5A3A3A3AE
:100B8700E00490029BF080289002D5E0FCA3E0FDF2
:100B9700A3E0FEA3E0FFE4FAF9F8EF2401FFEA3E41
:100BA700FEE93DFDE83CFC9002D5120E91020B04D4
:100BB7009002E4E025E0FF9002E3E033FE742C2F7F
:100BC700F582742A3EF583E493FE740193FF900245
:100BD7009BE0FDEFA805088005CEC313CE13D8F917
:100BE700FF900299EEF0A3EFF09002DBE0FEA3E0A6
:100BF700FF90029AE02FF0900299E03EF0E4251072
:100C0700FFE50F34F8FE9002D9F0A3EFF0FBAA0638
:100C1700EA3395E0F9F8900288E0FEA3E0FFEE33AF
:100C270095E0FDFC120E2C9002D1120E91E4FB7A96
:100C370008F9F89002D1E0FCA3E0FDA3E0FEA3E0F1
:100C4700FF1236AEE5122FFFE5113EFE9002A1F02E
:100C5700A3EFF0D394FFEE6480948F400A9002A133
:100C6700740FF0A374FFF0C39002A1E06480948036
:060C77005004E4F0A3F0BC
:010C7D002254
:1038A200A2AFE433FCC2AF758F0175B7A575B7F14E
:1038B2008F828E83EDF0E4F58FAF04EF24FF92AF99
:0138C20022E3
:10390500A2AFE433FDC2AF758F0375B7A575B7F1E7
:0F3915008F828E83E4F0F58FAF05EF24FF92AF22
:013924002280
:1035D700900376EEF0A3EFF0A3ECF0A3EDF0EB4A47
:1035E7006039900376E0FEA3E0FFA3E0FCA3E0F5DB
:1035F700828C83E0FD1238A2EB1B70011A900379CD
:10360700E004F07006900378E004F0900377E0049C
:0C361700F070CB900376E004F080C3223A
:083AB600E4900000F0A3F022EF
:1037F000900000E0FEA3E0FF123905900000E0FE1B
:10380000A3E0FF7C007D027B007A021235D7E490B2
:063810000000F0A3F0220D
:0A33A800A90590036AEEF0A3EFF010
:1033B200EE54FEFE900000E0FCA3E0FD7002EE6C15
:1033C2006057ED4C60031237F090036AE0FEEE5452
:1033D200FEFE7F00900000F0A3EFF090036CEEF091
:1033E200A3EFF0A37400F0A37402F07E0290036CCA
:1033F200E475F001120E1685F082F583E493FD90D8
:10340200036EE475F001120E1685F082F583EDF07D
:10341200EF1F70011EEF4E70D490036AE0FCA3E030
:10342200FDEC5401FC74022DF58274003CF583E935
:01343200F0A9
:013433002276
:1036230090035CEEF0A3EFF0A3EBF0A3EAF0A3E9C1
:10363300F090036174FFF5F0120E1645F0602690CA
:10364300035CE475F001120E16AFF0FE90035EE02A
:10365300FBA3E475F001120E16A9F0FA120D74FD26
:063663001233A880CC2206
:073AD40043C14053E6FE224E
:1018AD00900331E0FFA3E0FCA3E0FDA3E0FBA3E088
:1018BD00FAA3E0F9900304E513F0E514A3F0900307
:0618CD0039E0900306F073
:1018D3009002FEEFF0A3ECF0A3EDF0A3EBF0A3EA8C
:0418E300F0A3E9F095
:1018E7009003077403F0A374E8F0E5C120E5FBD289
:1018F700C1C2C4D2C5E4FF900394F030C0FDE5C077
:1019070054FE244070030219AA24FE602424E260D6
:101917000924FE600524E20219B2C2C5EF60030282
:1019270019B89002FEE025E044A0F5C27F03021932
:10193700B8EFB4030A9002FFE0F5C27F058072EFAB
:10194700B4050B9002FFA3E0F5C27F068063EF6446
:1019570006703E900306E0900301700FE0FBA3E4DE
:1019670075F001120E16A9F0FA8008E0FBA3E0FA61
:10197700A3E0F9120D74F5C2900305E024FFF0907F
:101987000304E034FFF0E07002A3E070247F0780D7
:1019970020EFB40706D2C47F09801690039474051C
:1019A700F0800E9003947402F08006900394740103
:1019B700F0EFB40904C2C08036900394E0FE6406D9
:1019C7006012EEB4021690030774FFF5F0120E00D2
:1019D70045F06008D2C5E4900394F0FF900394E0CB
:1019E7006008C2C5D2C4C2C08005C2C0021902E5E0
:0419F700C120E5FB2B
:0119FB0022C9
:102C4200900309EFF0A3ECF0A3EDF0A3EBF0A3EAFD
:042C5200F0A3E9F012
:102C56009003117403F0A374E8F0E5C120E5FBD2FC
:102C6600C1C2C4D2C5E4FF900394F030C0FDE5C0F4
:102C760054FE24C87003022D3324AE607A24CA7031
:102C860003022D3B24FE603824E2600924FE600521
:102C960024E2022D43C2C5EF700F900309E025E040
:102CA60044A0F5C27F03022D49EF64016003022DA3
:102CB60049900309E025E044A1F5C27F04022D49AD
:102CC600EFB4030A90030AE0F5C27F058075EFB4FE
:102CD600050B90030AA3E0F5C27F068066EFB406F3
:102CE60006D2C57F01805CEFB404047F0280549055
:102CF60003947405F0804C90030CE0FBA3E475F09C
:102D060001120E16A9F0FAE5C2120DBA900310E0F0
:102D160024FFF090030FE034FFF0E07002A3E070B0
:102D2600087F09C2C1D2C4801A7F0280169003941C
:102D36007406F0800E9003947402F080069003945B
:102D46007401F0EFB40904C2C08036900394E0FE2B
:102D560064066012EEB4021690031174FFF5F012C9
:102D66000E0045F06008D2C5E4900394F0FF90038E
:102D760094E06008C2C5D2C4C2C08005C2C0022C9D
:062D860071E5C120E5FB30
:012D8C002224
:102E9800900331EFF0900334EBF0A3EAF0A3E9F0EC
:082EA800900332ECF0A3EDF001
:102EB000751500543FF516543F605CC37440951679
:102EC000FFE49515FE900337E0FCA3E0FDC39FEC03
:102ED0009E50068C138D1480048E138F141218AD1F
:102EE000900394E060037F0222900333E02514F006
:102EF000900332E03513F0900339E0700B90033506
:102F0000E5138514F0120E00C3900338E09514F019
:102F1000900337E09513F0900337E0F513A3E0F545
:102F200014D3E5149400E51394004070E514944024
:102F3000E513940050131218AD900394E060037FE2
:102F40000222E4F513F51480D8900331E0FFA3E0EA
:102F5000FCA3E0FDA3E0FBA3E0FAA3E0F9900304E7
:102F6000E4F074401218C9900394E060037F0222D9
:102F700074C02514F51474FF3513F513900333E072
:102F80002440F0900332E03400F0900339E0709177
:0E2F900090033575F040120E00022F217F00D5
:012F9E002210
:103A350090030FE4F0A304F0122C42900394E0608D
:073A4500037F01227F002234
:1039B900900393EBF07B017A037993900337E4F05A
:0A39C900A304F0E4A3F0122E9822EC
:10388000C007900352E0FFA3E090030FCFF0A3EF37
:10389000F0D007122C42900394E060037F01227F56
:0238A000002204
:1039D300C00790035AE0FFA3E0900337CFF0A3EFB3
:0A39E300F0E4A3F0D007122E9822A2
:1034F900420262000042020D00004202080000C1BF
:0535090005C104C1032F
:0A3A9000C204C205E490020CF0220B
:10383B00E4900262F0A3F090020DF0A3F0A3F090DD
:10384B000208F0A3F0900203F0A37440F0E490029E
:03385B000BF0224D
:061A1B00123A9002383B74
:0D3A6B0075C19043E60190020A7401F0223B
:103A4C0043C140E5C120E5FB121A1BE490020AF0C9
:013A5C002247
:0A3A9A0053C1BF90020A7401F0222C
:0D3A7800AE07123A6B900207EEF0021A1B27
:10381600E4900391F0A3F0300402FF222005FDD2CC
:1038260004900205E4F0A37410F0900250EFF0E467
:04383600A3F07F017B
:01383A00226B
:1037650030040A900205E07002A3E070037F002296
:10377500900206E024FFF0900205E034FFF090028D
:1037850051E0FE04F074522EF582E43402F583EF25
:04379500F07F01229E
:0B3A8500300407C204D205123AA4224C
:0A3AA400E5C120E5FBC2C4D2C52233
:10343400900364EBF0A3EAF0A3E9F090020AE070D1
:1034440002FF22900367E0FE6005D3941040037FDF
:083454000022123816EF604E51
:10345C00E4900369F0900367E0FF900369E0FEC31A
:10346C009F5024900364E0FBA3E0FAA3E0F98E8262
:10347C00758300120D8DFF123765EF7002FF2290DD
:10348C000369E004F080CEE490020CF0123A8590CF
:0E349C000368E070032005FD90020CE0FF22A3
:0334AA007FFF227F
:0E2D8D0090037AEBF0A3EAF0A3E9F0A3EDF0D7
:102D9B00E4FFD3900263E09400900262E0648094BD
:102DAB008050012253E6FE900208E0FEA3E0240FC0
:102DBB00F58274023EF583E0FF900208E475F001A2
:102DCB00120E00FCE5F064404C7006900208F0A374
:102DDB00F0900204E004F07006900203E004F0E4CB
:102DEB00FE90037DE0FDEEC39D5054EEC39F504F0C
:102DFB00900208E0FCA3E0240FF58274023CF583FB
:102E0B00E0FD90037AE0FBA3E0FAA3E0F98E827574
:102E1B008300ED120DCC900208E475F001120E0048
:102E2B00FCE5F064404C7006900208F0A3F09002B1
:102E3B0004E004F07006900203E004F00E80A2EEB2
:102E4B00C39F5029900208E475F001120E00FCE5B7
:102E5B00F064404C7006900208F0A3F0900204E07E
:102E6B0004F07006900203E004F00E80D29002632F
:102E7B00E024FFF0900262E034FFF043E6019003A0
:0C2E8B007DE0FEEFC39E50028002AF0607
:012E97002218
:103A0500D3900263E09400900262E0648094804069
:083A1500047F0180027F002202
:031A18000215A014
:1015A000C0E0C0F0C083C082C0D075D000C000C011
:0315B00006C0076B
:1015B300C209E5C054FE120EDA168F08168F0A16FA
:1015C300560C16560E170810170812165C221667CB
:1015D3002816672A165C2C165C2E1649C01602C202
:1015E30015EDE015EDE200001713C203900250E081
:1015F300F5C2C2C5C2C490024F74FFF00217159022
:10160300024FE0FFB4FF12900251E0F5C2C2C5C21F
:10161300C490024FE4F0021715900251E0FEEFC3AD
:101623009E501790024FE0FF04F074522FF582E4AE
:101633003402F583E0F5C2021715D2C490020CE41C
:10164300F0C20502171590020C74FDF0D2C5C2C496
:1016530002171590024F74FFF0D203C2C4C2C1D265
:10166300C5021715E5C26007900207E0B5C20E90E8
:101673000202E4F0C2C5C2C4D2C1021715C2C4C279
:10168300C130030302170DC2C5021715900202E011
:101693007020E5C2F0E0FFC3900204E09F7480F87D
:1016A300900203E0648098500312383B900202E0FA
:1016B30004F0900204E024FFF0900203E034FFF012
:1016C30090020DE0FEA3E0240FF58274023EF58341
:1016D300E5C2F090020DE475F001120E00FEE5F094
:1016E30064404E700690020DF0A3F0900202E014E5
:1016F300F0700E900263E004F07006900262E00462
:10170300F0D2C1800DC2C4300308C203D2C5800227
:10171300D20930091053C17F43C180C2C5C2C4C2BC
:07172300C1C209C205C2C0EA
:10172A00D007D006D000D0D0D082D083D0F0D0E07D
:01173A00327C
:053AE200E5C15420FFC6
:013AE70022BC
:0E366900900370EBF0A3EAF0A3E9F0A3EDF0FC
:10367700E4900375F0900370E0FBA3E0FAA3E0F990
:10368700A3E0900367F0900374E0900368F0E4FF11
:10369700123434EFB4FF0D900375E0FE04F0EEC36F
:0636A700940340D17E00F7
:0136AD0022FA
:0B37990090038EEBF0A3EAF0A3E9F030
:1037A4007E007F007D10120F3190038EE0FBA3E0BA
:1037B400FAA3E0F97D10122D8DEF7002FF227F0134
:0137C40022E2
:103524009003137422F0A3EFF0A37413F0120D743C
:10353400900316F0900001120D8D900317F0900087
:1035440002120D8D900318F0900003120D8D90035C
:1035540019F0900004120D8D90031AF090000512DA
:103564000D8D90031BF0900006120D8D90031CF03E
:103574007B017A037913E4900374F07D0A023669BF
:1038C30090037E7422F0A3EFF0A37403F0A374FFBC
:1038D300F07B017A03797EE4900374F07D04023671
:0138E300697B
:1038E4009003827422F0A3EFF0A3741CF0A374FF7E
:1038F400F07B017A037982E4900374F07D0402364C
:013904006959
:10392500E4900386F0A3EFF0A3740AF0A3EFF07B15
:0F393500017A037986E4900374F07D0402366909
:0D350E004A031D0000000000000000000046
:0E102B0090FFFF120F00EFF090FFEE120F008B
:10103900851783851882E4F0A3F0900012120F241B
:10104900E025E0241DF582E43403F583E0FEA3E006
:10105900FFFBAA06E4F9F8900012120F24E075F0DC
:1010690002A424A6F582E5F03402F583E0FEA3E0AC
:10107900FFC3EF9BFFEE9AFEE499FDE498FC851708
:1010890083851882A3A3120E91E47F08FEFDFC85D7
:101099001783851882A3A3E0F8A3E0F9A3E0FAA3D4
:1010A900E0FBC3120E7B400B851783851882E4F0A1
:1010B900A304F074FF7FF8FEFDFC85178385188271
:1010C900A3A3E0F8A3E0F9A3E0FAA3E0FBD3120E8F
:1010D9007B500B85178385188274FFF0A3F0851761
:1010E90083851882E0FEA3E0FF4E7003021347EFE9
:0A10F900F47002EEF460030211E24D
:10110300900012120F24E025E0241DF582E434033D
:10111300F583E0FEA3E0FFE4FCFD90000E120F2434
:10112300120E91E47F01FEFDFC90000E120F24E0ED
:10113300F8A3E0F9A3E0FAA3E0FBC3120E7B500D82
:1011430090000E120F24120E9D0000000190001259
:10115300120F24E025E02409F8E6FE08E6FFE4FC8C
:10116300FD7BFF7A0FF9F8120E2C90000E120F245C
:10117300E0F8A3E0F9A3E0FAA3E0FB1236AE900097
:1011830006120F24120E91900012120F24E075F034
:1011930002A424A6F582E5F03402F583E0FEA3E081
:1011A300FFE4FCFD900006120F24E0F8A3E0F9A38E
:1011B300E0FAA3E0FB120E2C90000A120F24120E89
:1011C30091E47BFF7A0FF9F890000A120F24E0FCF8
:0C11D300A3E0FDA3E0FEA3E0FF1236AE97
:1011DF00021308851783851882E0FEA3E064014E91
:0511EF00600302131B68
:1011F400900012120F24E025E02409F8E6FE08E628
:10120400FBAA06C374FF9BFF740F9AFEE49400FDCF
:10121400E49400FCE47BFF7A0FF9F8120E2C9000A2
:1012240006120F24120E91900012120F24E025E0F2
:10123400241DF582E43403F583E0FEA3E0FBC374CC
:10124400FF9BFF740F9EFEE49400FDE49400FC9069
:10125400000A120F24120E91E47F01FEFDFC90009F
:101264000A120F24E0F8A3E0F9A3E0FAA3E0FBC319
:10127400120E7B500D90000A120F24120E9D0000D6
:101284000001900006120F24C083C082E0FCA3E09A
:10129400FDA3E0FEA3E0FF90000A120F24E0F8A3F0
:1012A400E0F9A3E0FAA3E0FB1236AED082D08312B9
:1012B4000E91900012120F24E075F002A424A6F5FA
:1012C40082E5F03402F583E0FEA3E0FBC374FF9BE8
:1012D400FF740F9EFEE49400FDE49400FC9000066D
:1012E400120F24E0F8A3E0F9A3E0FAA3E0FB120E46
:1012F4002CE47BFF7A0FF9F81236AEC374FF9FFF1C
:10130400740F9EFE900012120F24E025E02409F8C9
:07131400A60608A607D20798
:10131B00900012120F24E0FF75F002A424A6F582B0
:10132B00E5F03402F583E0FCA3E0FDEF25E0241D9E
:0C133B00F582E43403F583ECF0A3EDF040
:06134700900013020F00EC
:08351B00C106C1074102F100E5
:063AE800E49002F1F0225F
:073ADB009002F17401F022DA
:10331800E490038BF0A37403F0E4A3F0FE7F0BFDAD
:10332800FB7A007908120F31750B08750C00750FC0
:1033380008751000123AB67E7A7F017B017A03790C
:103348008C900361E4F0A304F0123623E490038A1E
:10335800F090038AE0FFC3941E502A75F00BEFA487
:103368002402F582E5F0347AAF82FE7B007A007998
:1033780008900361E4F0A3740BF012362390038ADB
:10338800E004F080CC1237F07E7A7F007B017A036C
:10339800798D900361E4F0A304F01236230237F02C
:103980003007199002A3E060132006109002F1E0C6
:0D39900070089002A4E0FF1238C3D2062296
:103A1D00907A00E493F46007A3E4936403600312C7
:083A2D003318E49002E5F022D9
:1037C5009002E5E0FFC3941E5020EF75F00BA42492
:1037D50002F9747A35F0FA7BFF78087C007D007E6B
:0B37E500007F0B120D4EC207C206222F
:103730009002E5E0C3941E502B123AB69002E5E0E9
:1037400075F00BA42402F582E5F0347AAF82FE7B9B
:10375000007A007908900361E4F0A3740BF012364C
:05376000231237F022E6
:083ABE00123730C207C20622D4
:05311E009002F3EDF04A
:103123009002F5E004F09002F8EFF0A3EBF09002C8
:10313300F3E0FF9002F8E0FED39F40030231D17524
:10314300F00BEEA42402F582E5F0347AAF8290020C
:10315300FAF0A3EFF09002F9E075F00BA42402F566
:1031630082E5F0347AAF829002FCF0A3EFF0E490B2
:1031730002F6F0A3F09002FCE475F001120E16AF14
:10318300F0FE9002FAE0FCA3E0F5828C83E493FD69
:103193001233A89002FBE004F070069002FAE004F8
:1031A300F09002F7E004F070069002F6E004F0C33A
:1031B3009002F7E0940B9002F6E0940040B71237C8
:0E31C300F09002F8E004F0A3E004F0023131D5
:0131D10022DB
:05173B0090033AEDF0FF
:1017400090033FEFF0A3EBF090033AE0FF90033FEC
:10175000E0D39F40030218ACA3E075F00BA4240271
:10176000F582E5F0347AAF8290033BF0A3EFF0E42A
:10177000900341F0A3F0900341E0FEA3E0FFC39487
:101780000BEE9400503890033BE0FCA3E0F5828C14
:1017900083E493FD74E62FF582E43402F583EDF0E3
:1017A00090033CE004F0700690033BE004F09003EB
:1017B00042E004F070C0900341E004F080B8900370
:1017C0003FE075F00BA42402F582E5F0347AAF8295
:1017D00090033DF0A3EFF0900340E075F00BA424DC
:1017E00002F582E5F0347AAF8290033BF0A3EFF08C
:1017F000E4900341F0A3F090033BE475F001120E76
:1018000016AFF0FE90033DE0FCA3E0F5828C83E48C
:1018100093FD1233A890033EE004F0700690033D60
:10182000E004F0900342E004F07006900341E0040D
:10183000F0C3900342E0940B900341E0940040B762
:1018400090033FE075F00BA42402F582E5F0347AB2
:10185000AF8290033DF0A3EFF0E4900341F0A3F0DA
:10186000900341E0FCA3E0FDC3940BEC9400502CEA
:1018700090033DE475F001120E16AFF0FE74E62DF4
:10188000F582E43402F583E0FD1233A8900342E0D0
:1018900004F070CC900341E004F080C41237F09063
:0C18A000033FE004F0A3E004F00217484E
:0118AC002219
:0B306800900327EFF0A3EDF0A3EBF0C6
:10307300A2AFE433A3F0C2AF123AD4900328E0FE28
:10308300900327E0FDEDFF90032FEEF0A3EFF0E4B4
:1030930090032BF0900329E0FF90032FE0FCA3E0C3
:1030A300FD7B017A0279E6900352E4F0A3740BF0FE
:1030B300123880900330E0240BF090032FE03400AB
:1030C300F090032BE075F00BA42402F9747A35F029
:1030D300FAA374FFF0A3EAF0A3E9F0123AB690035F
:1030E3002CA3E0FAA3E0AE02FF7B017A0279E6901B
:1030F3000361E4F0A3740BF01236231237F090034C
:103103002BE004F0E0C3941E408A9002A4E0FF1277
:0A3113003A7890032AE024FF92AFFF
:01311D00228F
:0B328200900343EFF0A3EDF0A3EBF08E
:10328D00A2AFE433A3F0C2AF123AD4900344E0FEF0
:10329D00900343E0FDEDFF900348EEF0A3EFF0E463
:1032AD00900347F0900347E0FFC3941E504C75F018
:1032BD000BEFA42402F582E5F0347AAF82FE900381
:1032CD004AF0FAA3EFF0FB900345E0FF900348E0CE
:1032DD00FCA3E0FDA9037BFF90035AE4F0A3740B5C
:1032ED00F01239D3900349E0240BF0900348E034F9
:1032FD0000F0900347E004F080AA9002A4E0FF12D2
:0A330D003A78900346E024FF92AFE7
:013317002293
:03000000020800F3
:03000300021A03DB
:03000B00021A06D0
:03001300021A09C5
:03001B00021A0CBA
:03002300021A0FAF
:03002B00021A12A4
:03003300021A1599
:03003B00021A188E
:03004300021A1B83
:03004B00021A1E78
:03005300021A216D
:03005B00021A2462
:03006300021A2757
:03006B00021A2A4C
:03007300021A2D41
:10080000E4F5D9E5EF7480F5FF7402F5EF787FE445
:10081000F6D8FD9000007F007E08E4F0A3DFFCDE48
:07082000FA75812102086254
:1008270002134DE493A3F8E493A34003F68001F287
:1008370008DFF48029E493A3F85407240CC8C333D2
:10084700C4540F4420C8834004F456800146F6DFA1
:10085700E4800B01020408102040809034ADE47E50
:10086700019360BCA3FF543F30E509541FFEE49396
:10087700A360010ECF54C025E060A840B8E493A35D
:10088700FAE493A3F8E493A3C8C582C8CAC583CA88
:10089700F0A3C8C582C8CAC583CADFE9DEE780BE40
:0135230000A7
:100C7E00E709F608DFFA8046E709F208DFFA803E58
:100C8E0088828C83E709F0A3DFFA8032E309F60845
:100C9E00DFFA8078E309F208DFFA807088828C83AD
:100CAE00E309F0A3DFFA806489828A83E0A3F60861
:100CBE00DFFA805889828A83E0A3F208DFFA804C3B
:100CCE0080D280FA80C680D4806980F28033801012
:100CDE0080A680EA809A80A880DA80E280CA80337B
:100CEE0089828A83ECFAE493A3C8C582C8CCC583F3
:100CFE00CCF0A3C8C582C8CCC583CCDFE9DEE780C3
:100D0E000D89828A83E493A3F608DFF9ECFAA9F041
:100D1E00EDFB2289828A83ECFAE0A3C8C582C8CC97
:100D2E00C583CCF0A3C8C582C8CCC583CCDFEADEB0
:100D3E00E880DB89828A83E493A3F208DFF980CC12
:100D4E0088F0EF60010E4E60C388F0ED2402B4040B
:100D5E000050B9F582EB2402B4040050AF232345B2
:060D6E008223900CCE73FD
:100D7400BB010689828A83E0225002E722BBFE027D
:090D8400E32289828A83E49322B0
:100D8D00BB010CE58229F582E5833AF583E022501B
:100D9D0006E92582F8E622BBFE06E92582F8E22265
:0D0DAD00E58229F582E5833AF583E493227F
:100DBA00BB010689828A83F0225002F722BBFE0118
:020DCA00F32212
:100DCC00F8BB010DE58229F582E5833AF583E8F05D
:100DDC00225006E92582C8F622BBFE05E92582C809
:020DEC00F222F1
:100DEE00EF8DF0A4A8F0CF8CF0A428CE8DF0A42E19
:020DFE00FE22D3
:100E0000C5F0F8A3E028F0C5F0F8E582158270027D
:060E10001583E038F0221A
:100E1600A3F8E0C5F025F0F0E5821582700215838F
:060E2600E0C838F0E822EC
:100E2C00E88FF0A4CC8BF0A42CFCE98EF0A42CFC65
:100E3C008AF0EDA42CFCEA8EF0A4CDA8F08BF0A4E3
:100E4C002DCC3825F0FDE98FF0A42CCD35F0FCEB42
:100E5C008EF0A4FEA9F0EB8FF0A4CFC5F02ECD3907
:0F0E6C00FEE43CFCEAA42DCE35F0FDE43CFC2274
:1036AE00C2D5E830E70FB2D5E4C39BFBE49AFAE447
:1036BE0099F9E498F8EC30E717B2D51236E4120F08
:1036CE0099E4C39BFBE49AFAE499F9E498F8800331
:1036DE00120F9930D50DE4C39FFFE49EFEE49DFDCD
:0436EE00E49CFC223A
:100E7B00EB9FF5F0EA9E42F0E99D42F0EC6480C8EE
:060E8B0064809845F0228E
:0C0E9100ECF0A3EDF0A3EEF0A3EFF022D4
:100E9D00A8828583F0D083D082120EB4120EB412C4
:100EAD000EB4120EB4E473E493A3C583C5F0C583E9
:100EBD00C8C582C8F0A3C583C5F0C583C8C582C89F
:010ECD002202
:0C0ECE00A42582F582E5F03583F583222F
:100EDA00D083D082F8E4937012740193700DA3A3A7
:100EEA0093F8740193F5828883E4737402936860BB
:060EFA00EFA3A3A380DFBB
:100F0000E5182582F582E5173583F583B517048545
:100F100082182210AF06858218F51722858218F5EF
:040F200017D2AF2213
:0D0F2400E5182582F582E5173583F5832257
:100F3100EF4E6012EF60010EEDBB010B89828A83D7
:100F4100F0A3DFFCDEFA2289F05007F709DFFCA9E4
:0C0F5100F022BBFEFCF309DFFCA9F0223B
:100F5D0075F008758200EF2FFFEE33FECD33CDCC4B
:100F6D0033CCC58233C5829BED9AEC99E5829840CE
:100F7D000CF582EE9BFEED9AFDEC99FC0FD5F0D6AB
:100F8D00E4CEFBE4CDFAE4CCF9A88222B800C1B9D5
:100F9D000059BA002DEC8BF084CFCECDFCE5F0CB13
:100FAD00F97818EF2FFFEE33FEED33FDEC33FCEB4C
:100FBD0033FB10D703994004EB99FB0FD8E5E4F907
:100FCD00FA227818EF2FFFEE33FEED33FDEC33FCF4
:100FDD00C933C910D7059BE99A4007EC9BFCE99AE8
:100FED00F90FD8E0E4C9FAE4CCFB2275F010EF2F2D
:100FFD00FFEE33FEED33FDCC33CCC833C810D7072D
:10100D009BEC9AE899400AED9BFDEC9AFCE899F867
:0E101D000FD5F0DAE4CDFBE4CCFAE4C8F922FA
:00000001FF
